:020000040000fa
:080000000002040000000000f2
:020000040000fa
:100400000f8d210000df23000001880000000000a4
:100410000c000700c0842300010020001100070029
:10042000000020000000e000020032000000020096
:10043000000000008a310200000000000040da00e5
:100440000000fe004440a900c0f820000000e000c9
:100450000300320000002000a00188004440a800f2
:100460000000060091018800800078000000eb0089
:1004700015003700e280400032a0b4009101ba00bc
:10048000e280400032a0b4009102ba00e280400055
:1004900032a0b4000002eb00472bde00f507b200eb
:1004a000602ce10004003a000059eb008301e900f0
:1004b000fdff3e00040037006128e100010032002a
:1004c0000082eb00040007001101ba000200e00006
:1004d000e8ff3a00000006003159ba008301e90044
:1004e0000c0032002159ba008301e90008003200f3
:1004f0000400e00003003a00e280400032a0b400b3
:10050000f5ff370011d9ba008301e900faff3a007c
:100510008100e800e180400032a0b4000000060045
:1005200003f0a200889fbe008a9fbe008c1f780047
:10053000930107009a0133006450e1004f0032003c
:100540006420e1005200320003826c0007003b008f
:100550000905d0000306d000820f54000c065d0090
:100560000200390002003200890178000306780099
:100570008582550004003d000003fd008103fd005d
:100580008502ea008b854200840f720002003b0066
:1005900060001000e08018006011b8000005eb005a
:1005a0007a28e1000a00390006007800c75ddd0006
:1005b000f707b200878075002d0037008281710037
:1005c0000a017800610560008180d1000080d300bd
:1005d0008502e900f9ff3b000604400087844800db
:1005e00002003b0060041400e0841c000988a300a2
:1005f000070032008a81710082817100610164000c
:100600008904d1000884d3008b05e8001700370067
:100610000978a30013003a000b00e0001300340037
:100620008b05e9000804440089844c000a447400e6
:100630000978a3000d003a000b00e0000700340029
:100640008b05e9000804440089844c0001003a004d
:100650000b0020000978a300f7ff32000001eb0037
:1006600002003700828171000a0178005c010700f6
:100670000cf0a70001f0a000520137006420e10057
:1006800002003a00838f6c00520133000801be0063
:100690000200be004b013700889fbe008a9fbe004b
:1006a0008c1f7800360107003d01330003866c0083
:1006b0006450e100240032006420e1002700320091
:1006c0006150e100220032006120e100210032008f
:1006d0008b854200eb07b1000134b800003ab80046
:1006e0000804420089844a00013ab8000030b8008a
:1006f0008880400009014a000400330000004000e7
:1007000081804800020149008b05e900c909dd002c
:10071000830170000100320013002000c814de00c5
:100720004814dd004709de001200b200c808de00f0
:10073000088470002a01070001f0a1000cf0a70056
:1007400001f0a0001f0137006120e100210132000b
:100750000801be000200be00f7ff37006150e10053
:10076000fcff3a001b0137000001be0042010700f8
:100770000470a70003f0a1006509b1001600320063
:100780000d0035006828e10006003500f0ff2f005d
:10079000f1ff27000300e00013003b0001002800e8
:1007a0000000050000004000818048008502e9004b
:1007b000fcff3a0008003700f88f420002003c00be
:1007c0008000eb00000005008100d1000080d30014
:1007d0008502e800fcff3a000300e00002003b0055
:1007e00060001000e080180000000600889fbe0036
:1007f0008a9fbe00010578000100e000040035007a
:1008000008003c000000e000200032000500370036
:1008100060001000e080180002003b0001f02c0096
:100820001a0037000004be006011b8006b092000f8
:100830000982cf00020039000882cf000441b000d5
:10084000694252000e00320008003b0082817100b4
:10085000610164008904d1000884d3008b05e8009d
:100860000442e800f9ff3a0005003700080444009c
:1008700089844c008b05e9000442e900fbff3a0043
:10088000d70007000af0a70001f0a0004f05be0046
:100890004f04be00000006000001be00f600070085
:1008a0000470a70003f0a10003f8a30013003a00ae
:1008b0006509b10010003200090035006928e10027
:1008c0000200350001002800000005000000400083
:1008d000818048008502e900fcff3a000000060024
:1008e000f88f4200050035008100d1000080d30060
:1008f0008502e800fcff3a00000006008000eb00e3
:1009000000000500889fbe008a9fbe008c1f7800f3
:100910009b000700a200330003866c006450e100d6
:100920002e0032006420e100330032006150e1000b
:100930002f0032006120e100310032008585550032
:10094000eb07b00009002000080420000500370074
:100950000804440089844c000a0031000603430067
:1009600087834b000001530081815b00f8ff330057
:100970000203be000800a0000804440089844c0063
:10098000f6ff3900c639dd00830173000100320033
:10099000130020008904d1000884d3000998a30023
:1009a000050032000800a7000300a0008904d10060
:1009b0000884d3008b05e8008904d1000884d300a3
:1009c0000001eb000281d2008500070001f0a100c8
:1009d0000cf0a70001f0a0007a0037006420e100cd
:1009e0007c0032000801be000200be00f7ff3700a5
:1009f0006120e100770032006000b800f3ff3700ab
:100a00000000200001f82700f0ff3700889fbe009b
:100a10008a9fbe008c9fbe00ac0007008504780052
:100a20000005be006420e10049003e006220e100b4
:100a300003003200090035000bf8a3004400320027
:100a40000bf8a300080032001002200070c68800d6
:100a5000f0ff2f00f1ff27003d00370001f82f00c5
:100a6000000020003a0037003d000700acfe070000
:100a70000006be000a00be00324f200053f32300e0
:100a80003d000700060034000c00be0034000700e3
:100a9000a3fe07000006be000a00be0002003700e9
:100aa0008904e9000c00be002d000700fafe0700d3
:100ab0002b0007009bfe07000001be000c00be00db
:100ac00090ff07000005be000001be00f2fe070017
:100ad0000006be00a2f32300430d2c0091fe070088
:100ae000809fbe000c00be00d2e32700d3f02b0095
:100af000e9fe07004f01be0082ff07000006be00ae
:100b00000a01be00e4fe07000a01be0085fe0700e0
:100b10000006be006148b90034ff07000005be00b2
:100b200032082800e3952b00dbfe07000c01be0015
:100b30007cfe07000006be000a00be00020028007e
:100b400013f32300d4fe07000c01be0075fe07005e
:100b50004f06be004f05be004f04be000000060059
:100b600003f0230002000500a8ff070092bd250046
:100b7000e3ed2300c8fe3700f4ff2f0060003700cc
:100b80000004be003c0007000003be000405be00d8
:100b90000200be0038000700844f75000000060008
:100ba0000200be006450e100050036006420e10050
:100bb000020036000968a30001003a000800be00e8
:100bc0000160a0004f0678004f05be004f04be0034
:100bd00000000600f0ff2f00f1ff2700f9ff3700ab
:100be00081002000618055000b003d000b002000bb
:100bf00061fe2f000100e1001d00340082817100c0
:100c0000610164008904d1000884d3000000e80079
:100c1000faff3a00710020006100640003007000d8
:100c2000020060000900320061044400e0844c00ce
:100c30000988a500050032008b05e8006808e1007e
:100c400002003a008904d1000884d300f20f20008a
:100c50000258e10005003d00c75ddd00f907b20064
:100c60008980750008007800000006000bf8270056
:100c70008b00780000000500c70ade00f107b20013
:100c8000f50fb20008003200e1cf4200020032004e
:100c90000170a00024000500810f700001003200e7
:100ca0000408050044000500810f700002003a00ae
:100cb000140005008502e9000000400081c04800e2
:100cc000fcff3b000170a000240005000003be00f3
:100cd000e9ff07006220e100020032000600be00ca
:100ce00005000500e507b100f107b20004f023009c
:100cf0008480700007f0a70001f0a0002400050028
:100d0000889fbe008a9fbe00841f78009cff07005a
:100d10004f00780011003300f0ff2f00838f6c002c
:100d200006003b00040565000a00a7000800370024
:100d300009f0a6001000200008003700820f5400c0
:100d4000838f5c00030039001000200001003e008a
:100d50000000200009f0a7000000ea004f05be00d7
:100d60004f04be000000e00000000600889fbe00a7
:100d70008a9fbe008c9fbe004400f800070f200031
:100d8000270288003400f80007f02f000338e10044
:100d900004003200270280004700b30027028800c9
:100da000a3018800811f780019002000804cdd001d
:100db0001300200002047800800678008904d10026
:100dc000424edd00010578000302e90004800800be
:100dd000170000008a0546004218dd000902e900fc
:100de0000480080010000000000000004620c3003e
:100df0003b025200df35c100080440001381c200ed
:100e0000ab825200264dc5003e85c400bb00cd001c
:100e1000bb80cd003a00ca002a80ca000700c90082
:100e20000580c900ba00cd00ba80cd000a05460091
:100e3000020478008301d0008d06e900dfff3c004a
:100e40004f0078003400f9004400f9004f06be005e
:100e50004f05be004f04be00000006004600f8002b
:100e60005000f80002202000320288000200280012
:100e7000130020008019dd000281710082028800c9
:100e800001007800010178002600200047002000c2
:100e90008301e90003800800070000000110e10061
:100ea000040034001102be0092087800e2307b009a
:100eb0000489be0087804000121978005000f900b4
:080ec0004600f90000000600e5
:020000040000fa
:0200000401f009
:04000000ffff0000fe
:020000040000fa
:0200000401f009
:04000400ffff0000fa
:020000040000fa
:0200000401f009
:04000800ffff0000f6
:020000040000fa
:0200000401f009
:04000c00f8ff0000f9
:020000040000fa
:0200000401f009
:040010007eff00006f
:020000040000fa
:0200000401f009
:040014007fff00006a
:020000040000fa
:0200000401f009
:04001800fdff0000e8
:020000040000fa
:0200000401f009
:04001c00dfff000002
:020000040000fa
:10000800ba390000ba390000ba390000ba3900001c
:10001800ba390000ba390000ba390000ba3900000c
:10002800ba390000ba390000ba39000002390000b4
:10003800ba390000ba390000ba390000ba390000ec
:10004800ba390000ba390000ba390000ba390000dc
:10005800ba390000ba390000ba390000ba390000cc
:10006800ba390000ba390000ba3900009e390000d8
:10007800ba390000ba390000ba390000ba390000ac
:10008800ba390000ba390000ba390000ba3900009c
:10009800ba390000ba390000ba390000ba3900008c
:1000a800ba390000ba390000ba390000ba3900007c
:1000b800ba390000ba390000ba390000ba3900006c
:1000c800ba390000ba390000ba390000ba3900005c
:1000d800ba390000ba390000ba390000ba3900004c
:1000e800ba390000ba390000ba390000ba3900003c
:1000f800ba390000ba390000ba390000ba3900002c
:10010800ba390000ba390000ba390000ba3900001b
:10011800e22c0000ba390000ba390000ba390000f0
:10012800ba390000ba390000ba390000ba390000fb
:10013800ba390000ba390000ba390000ba390000eb
:10014800ba390000ba390000ba390000ba390000db
:10015800ba390000ba390000ba390000ba390000cb
:10016800ba390000ba390000ba390000ba390000bb
:10017800ba390000ba390000ba390000ba390000ab
:10018800ba390000ba390000ba390000ba3900009b
:10019800ba390000ba390000ba390000ba3900008b
:1001a800ba390000ba390000ba390000ba3900007b
:1001b800ba390000ba390000ba390000ba3900006b
:1001c800ba390000ba390000ba390000ba3900005b
:1001d800ba390000ba390000ba390000ba3900004b
:1001e800ba390000ba390000ba390000ba3900003b
:0801f800ba390000ba39000019
:020000040000fa
:10020800ba390000ba390000ba390000ba3900001a
:10021800ba390000ba390000ba390000ba3900000a
:10022800ba390000ba390000ba39000002390000b2
:10023800ba390000ba390000ba390000ba390000ea
:10024800ba390000ba390000ba390000ba390000da
:10025800ba390000ba390000ba390000ba390000ca
:10026800ba390000ba390000ba3900009e390000d6
:10027800ba390000ba390000ba390000ba390000aa
:10028800ba390000ba390000ba390000ba3900009a
:10029800ba390000ba390000ba390000ba3900008a
:1002a800ba390000ba390000ba390000ba3900007a
:1002b800ba390000ba390000ba390000ba3900006a
:1002c800ba390000ba390000ba390000ba3900005a
:1002d800ba390000ba390000ba390000ba3900004a
:1002e800ba390000ba390000ba390000ba3900003a
:1002f800ba390000ba390000ba390000ba3900002a
:10030800ba390000ba390000ba390000ba39000019
:10031800e22c0000ba390000ba390000ba390000ee
:10032800ba390000ba390000ba390000ba390000f9
:10033800ba390000ba390000ba390000ba390000e9
:10034800ba390000ba390000ba390000ba390000d9
:10035800ba390000ba390000ba390000ba390000c9
:10036800ba390000ba390000ba390000ba390000b9
:10037800ba390000ba390000ba390000ba390000a9
:10038800ba390000ba390000ba390000ba39000099
:10039800ba390000ba390000ba390000ba39000089
:1003a800ba390000ba390000ba390000ba39000079
:1003b800ba390000ba390000ba390000ba39000069
:1003c800ba390000ba390000ba390000ba39000059
:1003d800ba390000ba390000ba390000ba39000049
:1003e800ba390000ba390000ba390000ba39000039
:0803f800ba390000ba39000017
:020000040000fa
:100ec80000000000320000006400000096000000ee
:100ed800c9000000fb0000002d0100005f010000b8
:100ee80092010000c4010000f60100002802000081
:100ef8005b0200008d020000bf020000f10200004a
:100f0800240300005603000088030000ba03000011
:100f1800ed0300001f0400005104000083040000da
:100f2800b6040000e80400001a0500004c050000a3
:100f38007e050000b1050000e3050000150600006d
:100f4800470600007a060000ac060000de06000036
:100f5800100700004207000074070000a707000000
:100f6800d90700000b0800003d0800006f080000ca
:100f7800a1080000d4080000060900003809000094
:100f88006a0900009c090000ce090000000a000060
:100f9800320a0000650a0000970a0000c90a00002a
:100fa800fb0a00002d0b00005f0b0000910b0000f6
:100fb800c30b0000f50b0000270c0000590c0000c3
:100fc8008b0c0000bd0c0000ef0c0000210d000090
:100fd800530d0000850d0000b70d0000e90d00005d
:100fe8001b0e00004d0e00007f0e0000b10e000029
:100ff800e30e0000150f0000470f0000790f0000f6
:10100800ab0f0000dc0f00000e10000040100000c5
:1010180072100000a4100000d61000000711000094
:10102800391100006b1100009d110000cf11000064
:101038000012000032120000641200009612000034
:10104800c7120000f91200002b1300005d13000006
:101058008e130000c0130000f213000023140000d8
:101068005514000086140000b8140000ea140000ab
:101078001b1500004d1500007e150000b01500007e
:10108800e115000013160000441600007616000053
:10109800a7160000d91600000a1700003c17000028
:1010a8006d1700009f170000d017000001180000fe
:1010b800331800006418000095180000c7180000d5
:1010c800f8180000291900005b1900008c190000ad
:1010d800bd190000ee190000201a0000511a000086
:1010e800821a0000b31a0000e41a0000151b000061
:1010f800461b0000781b0000a91b0000da1b00003b
:101108000b1c00003c1c00006d1c00009e1c000015
:10111800cf1c0000001d0000311d0000621d0000f2
:10112800931d0000c31d0000f41d0000251e0000d3
:10113800561e0000871e0000b81e0000e81e0000b2
:10114800191f00004a1f00007b1f0000ab1f000092
:10115800dc1f00000d2000003d2000006e20000074
:101168009f200000cf200000002100003021000057
:101178006121000091210000c2210000f22100003d
:10118800232200005322000084220000b422000021
:10119800e422000015230000452300007523000009
:1011a800a6230000d62300000624000036240000f1
:1011b8006724000097240000c7240000f7240000db
:1011c800272500005725000087250000b7250000c7
:1011d800e7250000172600004726000077260000b4
:1011e800a7260000d72600000727000037270000a1
:1011f8006727000097270000c6270000f627000091
:10120800262800005628000085280000b528000080
:10121800e528000014290000442900007329000073
:10122800a3290000d2290000022a0000312a000068
:10123800612a0000902a0000c02a0000ef2a00005e
:101248001e2b00004e2b00007d2b0000ac2b000055
:10125800db2b00000b2c00003a2c0000692c00004e
:10126800982c0000c72c0000f62c0000252d00004b
:10127800542d0000832d0000b22d0000e12d000048
:10128800102e00003f2e00006e2e00009d2e000044
:10129800cc2e0000fa2e0000292f0000582f000045
:1012a800862f0000b52f0000e42f00001230000048
:1012b800413000006f3000009e300000cc3000004c
:1012c800fb30000029310000583100008631000051
:1012d800b4310000e3310000113200003f32000059
:1012e8006d3200009c320000ca320000f832000063
:1012f800263300005433000082330000b03300006e
:10130800de3300000c3400003a340000683400007a
:1013180096340000c3340000f13400001f3500008b
:101328004d3500007a350000a8350000d63500009c
:1013380003360000313600005e3600008c360000af
:10134800b9360000e73600001437000041370000c6
:101358006f3700009c370000c9370000f6370000df
:1013680024380000513800007e380000ab380000f7
:10137800d838000005390000323900005f39000014
:101388008c390000b9390000e6390000123a000033
:101398003f3a00006c3a0000993a0000c53a000054
:1013a800f23a00001f3b00004b3b0000783b000076
:1013b800a43b0000d13b0000fd3b0000293c00009d
:1013c800563c0000823c0000ae3c0000db3c0000c4
:1013d800073d0000333d00005f3d00008b3d0000ed
:1013e800b73d0000e33d00000f3e00003b3e00001b
:1013f800673e0000933e0000bf3e0000eb3e000049
:10140800163f0000423f00006e3f0000993f000079
:10141800c53f0000f03f00001c40000047400000ae
:10142800734000009e400000ca400000f5400000e4
:10143800204100004c41000077410000a24100001b
:10144800cd410000f8410000234200004e42000058
:1014580079420000a4420000cf420000fa42000096
:1014680025430000504300007a430000a5430000d4
:10147800d0430000fa430000254400004f44000018
:101488007a440000a4440000cf440000f94400005e
:10149800234500004e45000078450000a2450000a5
:1014a800cc450000f6450000204600004a460000f2
:1014b800744600009e460000c8460000f246000040
:1014c8001c470000464700006f470000994700008e
:1014d800c3470000ec470000164800003f480000e2
:1014e8006948000092480000bc480000e548000038
:1014f8000e49000038490000614900008a4900008f
:10150800b3490000dc490000054a00002e4a0000eb
:10151800574a0000804a0000a94a0000d24a000049
:10152800fa4a0000234b00004c4b0000744b0000ab
:101538009d4b0000c54b0000ee4b0000164c000010
:101548003f4c0000674c00008f4c0000b84c000076
:10155800e04c0000084d0000304d0000584d0000e0
:10156800804d0000a84d0000d04d0000f84d00004f
:10157800204e0000484e00006f4e0000974e0000bd
:10158800bf4e0000e64e00000e4f0000354f000031
:101598005d4f0000844f0000ac4f0000d34f0000a7
:1015a800fa4f000021500000495000007050000020
:1015b80097500000be500000e55000000c5100009c
:1015c800335100005951000080510000a75100001c
:1015d800ce510000f45100001b520000415200009f
:1015e800685200008e520000b5520000db52000025
:1015f80001530000285300004e53000074530000ac
:101608009a530000c0530000e65300000c54000039
:1016180032540000585400007d540000a3540000c8
:10162800c9540000ef540000145500003a5500005a
:101638005f55000085550000aa550000cf550000f1
:10164800f45500001a5600003f560000645600008a
:1016580089560000ae560000d3560000f856000028
:101668001d57000042570000665700008b570000c6
:10167800b0570000d4570000f95700001d5800006b
:1016880042580000665800008a580000af58000011
:10169800d3580000f75800001b5900003f590000bc
:1016a8006359000087590000ab590000cf5900006a
:1016b800f3590000165a00003a5a00005e5a00001a
:1016c800815a0000a55a0000c85a0000ec5a0000d0
:1016d8000f5b0000325b0000565b0000795b000086
:1016e8009c5b0000bf5b0000e25b0000055c000043
:1016f800285c00004b5c00006d5c0000905c000002
:10170800b35c0000d65c0000f85c00001b5d0000c4
:101718003d5d00005f5d0000825d0000a45d00008b
:10172800c65d0000e95d00000b5e00002d5e000054
:101738004f5e0000715e0000935e0000b45e000022
:10174800d65e0000f85e00001a5f00003b5f0000f4
:101758005d5f00007e5f0000a05f0000c15f0000c9
:10176800e25f0000046000002560000046600000a1
:101778006760000088600000a9600000ca6000007f
:10178800eb6000000c6100002d6100004d6100005d
:101798006e6100008e610000af610000cf61000043
:1017a800f061000010620000306200005162000029
:1017b8007162000091620000b1620000d162000015
:1017c800f162000011630000306300005063000004
:1017d800706300008f630000af630000ce630000f9
:1017e800ee6300000d6400002d6400004c640000ee
:1017f8006b6400008a640000a9640000c8640000eb
:10180800e7640000066500002565000044650000e7
:101818006265000081650000a0650000be650000eb
:10182800dd650000fb6500001966000038660000f1
:10183800566600007466000092660000b0660000fc
:10184800ce660000ec6600000a670000286700000a
:101858004567000063670000816700009e6700001d
:10186800bc670000d9670000f76700001468000033
:10187800316800004e6800006b680000886800004e
:10188800a5680000c2680000df680000fc6800006e
:101898001969000035690000526900006e6900008e
:1018a8008b690000a7690000c4690000e0690000b6
:1018b800fc690000186a0000346a0000506a0000e1
:1018c8006c6a0000886a0000a46a0000c06a000010
:1018d800db6a0000f76a0000136b00002e6b000043
:1018e8004a6b0000656b0000806b00009c6b000079
:1018f800b76b0000d26b0000ed6b0000086c0000b5
:10190800236c00003e6c0000586c0000736c0000f3
:101918008e6c0000a86c0000c36c0000dd6c000039
:10192800f86c0000126d00002c6d0000476d00007f
:10193800616d00007b6d0000956d0000af6d0000cb
:10194800c96d0000e36d0000fc6d0000166e00001c
:10195800306e0000496e0000636e00007c6e00006f
:10196800956e0000af6e0000c86e0000e16e0000ca
:10197800fa6e0000136f00002c6f0000456f000026
:101988005e6f0000766f00008f6f0000a86f000088
:10199800c06f0000d96f0000f16f000009700000ef
:1019a800227000003a700000527000006a70000057
:1019b800827000009a700000b2700000ca700000c7
:1019c800e1700000f970000011710000287100003a
:1019d80040710000577100006e71000086710000b0
:1019e8009d710000b4710000cb710000e27100002d
:1019f800f971000010720000267200003d720000ac
:101a0800547200006a720000817200009772000030
:101a1800ae720000c4720000da720000f0720000ba
:101a2800067300001c730000327300004873000046
:101a38005e73000074730000897300009f730000d8
:101a4800b5730000ca730000df730000f57300006f
:101a58000a7400001f740000347400004974000008
:101a68005e74000073740000887400009d740000a8
:101a7800b1740000c6740000db740000ef7400004d
:101a880003750000187500002c75000040750000f3
:101a980054750000687500007c75000090750000a2
:101aa800a4750000b8750000cc750000df75000053
:101ab800f3750000067600001a7600002d76000007
:101ac8004076000053760000677600007a760000c2
:101ad8008d760000a0760000b2760000c576000082
:101ae800d8760000ea760000fd7600001077000046
:101af800227700003477000047770000597700000c
:101b08006b7700007d7700008f770000a1770000d9
:101b1800b3770000c4770000d6770000e8770000ac
:101b2800f97700000b7800001c7800002e78000080
:101b38003f7800005078000061780000727800005b
:101b48008378000094780000a5780000b67800003b
:101b5800c6780000d7780000e7780000f878000021
:101b68000879000019790000297900003979000006
:101b780049790000597900006979000079790000f5
:101b88008979000098790000a8790000b8790000e8
:101b9800c7790000d7790000e6790000f5790000e0
:101ba800047a0000147a0000237a0000327a0000d8
:101bb800417a00004f7a00005e7a00006d7a0000da
:101bc8007c7a00008a7a0000997a0000a77a0000df
:101bd800b57a0000c47a0000d27a0000e07a0000ea
:101be800ee7a0000fc7a00000a7b0000187b0000f7
:101bf800257b0000337b0000417b00004e7b00000a
:101c08005c7b0000697b0000767b0000837b000022
:101c1800917b00009e7b0000ab7b0000b87b00003e
:101c2800c47b0000d17b0000de7b0000eb7b000062
:101c3800f77b0000047c0000107c00001c7c000086
:101c4800297c0000357c0000417c00004d7c0000b0
:101c5800597c0000657c0000707c00007c7c0000e2
:101c6800887c0000937c00009f7c0000aa7c000018
:101c7800b67c0000c17c0000cc7c0000d77c000052
:101c8800e27c0000ed7c0000f87c0000037d000091
:101c98000e7d0000187d0000237d00002e7d0000d1
:101ca800387d0000427d00004d7d0000577d00001a
:101cb800617d00006b7d0000757d00007f7d000068
:101cc800897d0000937d00009c7d0000a67d0000ba
:101cd800b07d0000b97d0000c27d0000cc7d000011
:101ce800d57d0000de7d0000e77d0000f07d00006e
:101cf800f97d0000027e00000b7e0000137e0000cc
:101d08001c7e0000257e00002d7e0000367e00002f
:101d18003e7e0000467e00004e7e0000567e00009b
:101d28005e7e0000667e00006e7e0000767e00000b
:101d38007e7e0000857e00008d7e0000947e00007f
:101d48009c7e0000a37e0000aa7e0000b27e0000f8
:101d5800b97e0000c07e0000c77e0000ce7e000075
:101d6800d47e0000db7e0000e27e0000e87e0000fa
:101d7800ef7e0000f57e0000fc7e0000027f000080
:101d8800087f00000e7f0000147f00001a7f00000b
:101d9800207f0000267f00002c7f0000317f00009c
:101da800377f00003c7f0000427f0000477f000033
:101db8004c7f0000527f0000577f00005c7f0000ce
:101dc800617f0000667f00006a7f00006f7f00006f
:101dd800747f0000787f00007d7f0000817f000015
:101de800867f00008a7f00008e7f0000927f0000bf
:101df800967f00009a7f00009e7f0000a27f00006f
:101e0800a67f0000a97f0000ad7f0000b07f000022
:101e1800b47f0000b77f0000bb7f0000be7f0000da
:101e2800c17f0000c47f0000c77f0000ca7f000098
:101e3800cd7f0000cf7f0000d27f0000d57f00005b
:101e4800d77f0000d97f0000dc7f0000de7f000024
:101e5800e07f0000e27f0000e47f0000e67f0000f2
:101e6800e87f0000ea7f0000ec7f0000ee7f0000c2
:101e7800ef7f0000f17f0000f27f0000f37f000099
:101e8800f57f0000f67f0000f77f0000f87f000074
:101e9800f97f0000fa7f0000fb7f0000fb7f000055
:101ea800fc7f0000fd7f0000fd7f0000fe7f00003a
:101eb800fe7f0000fe7f0000fe7f0000fe7f000026
:101ec800ff7f000000000000efff0000040000009a
:101ed80002000000e5ff0000e1ff0000fcff000039
:101ee800faff0000d4ff0000cfff0000f7ff00005a
:101ef800f8ff0000c3ff0000c0ff00000000000062
:101f080006000000bfff0000c1ff00002500000020
:101f180035000000d4ff0000ddff00007100000064
:101f28008a000000000000000c000000d80000003b
:101f3800f30000002c000000310000003701000011
:101f48004901000027000000160000005b010000a6
:101f580057010000b8ff000085ff000019010000cc
:101f6800f8000000b9fe000062fe00006c000000ee
:101f78003700000038fd0000c8fc000093ff000097
:101f880066ff000078fb00000afb00001cff000051
:101f980029ff0000eef90000a2f90000000000008f
:101fa800a200000016f9000005f900007304000003
:101fb800e706000043f9000079f90000a41c0000be
:101fc800ff3f00006f310000f7fa000094d80000ce
:101fd800d0e4000091fc000024fd00004ef2000057
:101fe8009bf40000e7fe000075ff000061f90000a7
:101ff8008ffa0000f50000005e01000043fd0000bc
:10200800f2fd00004e020000800200006aff00009e
:10201800bfff0000c7020000c40200004e0000001d
:102028006300000080020000580200005b0000000e
:102038004b000000c70100009201000000000000f2
:10204800e6ff0000f9000000ca0000009bff000046
:1020580088ff0000580000003a00000063ff0000fd
:102068005fff000000000000f5ff000064ff0000b3
:102078006cff0000e9ff0000eaff00008cff000091
:1020880099ff0000f6ff0000faff0000beff000005
:10209800c9ff0000090000000d000000e4ff000077
:1020a800ecff00001600000017000000faff000017
:1020b800feff00001a0000001a00000002000000e5
:1020c8000000000000000000fcff0000fdff000011
:1020d800e5ff0000e6ff0000020000000500000028
:1020e800e8ff0000eaff0000140000001b000000e9
:1020f800f3ff0000f6ff0000360000004200000079
:10210800050000000a0000006700000074000000dd
:102118001600000016000000930000009b0000005d
:102128000a000000ffff0000a00000009c00000063
:10213800c5ff0000a8ff0000770000006500000050
:1021480036ff000007ff00001a0000000000000032
:102158006efe000038fe0000b5ff0000a4ff00007e
:10216800a8fd000080fd00009dff0000b1ff0000f9
:102178003cfd000038fd0000410000009600000012
:1021880080fd0000b2fd00000e020000bd0200004c
:10219800a2fe00000aff0000700500009e06000075
:1021a8008a00000018010000650b0000b10d000056
:1021b800dc0200006e0300002f1b00006b270000ec
:1021c8000905000091ce000001c000005be300009b
:1021d80086060000bc06000018f900008cfb000011
:1021e800fb060000ea0600005dff0000000000009a
:1021f8005e06000011060000d6000000e3000000a3
:10220800f504000087040000990000006c0000003d
:1022180037030000c8020000c9ff000094ff000057
:102228009d0100004601000008ff0000e7fe0000d5
:102238007b00000048000000a9fe0000a4fe00008a
:10224800eaff0000d9ff0000b7fe0000c8fe00004a
:10225800ceff0000d3ff00000cff000028ff0000a5
:10226800f3ff0000ffff000076ff00008fff000073
:10227800230000002c000000caff0000daff000065
:102288003f00000041000000f9ff000000000000ce
:10229800400000003d0000000800000008000000a9
:1022a800300000002b0000000500000004000000c2
:1022b8001e0000001a000000feff0000fcff0000e6
:1022c8000000000080ff00007aff000081ff00008e
:1022d80095ff0000b6ff0000e4ff00001c000000ae
:1022e8005900000094000000c7000000e900000049
:1022f800f5000000e5000000bb0000007a000000c7
:102308002a000000d7ff00008eff00005bff0000de
:1023180048ff000057ff000084ff0000c1ff0000d5
:10232800fdff0000220000001a000000d5ff000099
:102338004dff00008afe0000a4fd0000c1fc000063
:1023480010fc0000c6fb000011fc000014fd00009a
:10235800d8fe00004b0100003b04000058070000b5
:102368003c0a0000760c00009b0d0000530d000095
:102378006b0b0000e1070000e8020000ebfc000026
:1023880082f6000066f0000056eb000004e800004a
:10239800fce600008de80000bbec00003cf3000008
:1023a80079fb0000a0040000b90d0000c215000070
:1023b800d11b00002f1f00006f1f00007e1c0000b3
:1023c800a6160000840e0000fa0400000ffb0000af
:1023d800d2f100003cea00000ee50000c1e2000076
:1023e80076e30000f5e60000bdec00000ff4000005
:1023f8000bfc0000cd030000890a00009c0f0000c0
:10240800a31200007e13000050120000730f00009a
:10241800690b0000c80600002602000005fe000047
:10242800c7fa0000a5f80000aef70000c9f70000e1
:10243800bff8000047fa000013fc0000d9fd0000b7
:1024480061ff0000840000003301000075010000f6
:102458005f0100000e010000a6000000440000001b
:10246800fdff0000e0ff0000ecff00001a00000084
:102478005d000000a4000000df0000000301000070
:1024880008010000ef000000bb000000740000001d
:1024980026000000daff00009aff00006aff000033
:1024a8004fff000049ff000055ff000070ff0000cb
:1024b80095ff0000bfff0000ebff000014000000c4
:1024c8000102000004080000102000004080000005
:1024d80000800000c0e00000f0f80000fcfe0000f2
:1024e800000000000000000000000000005f000085
:1024f80000000000000700000007000000140000b2
:102508007f1400007f140000242a00007f2a0000a6
:10251800122300001308000064620000364900001e
:1025280055220000500000000503000000000000d4
:10253800001c0000224100000000000041220000b1
:102548001c000000082a00001c2a000008080000df
:10255800083e00000808000000500000300000009d
:1025680000080000080800000808000000600000db
:1025780060000000002000001008000004020000b5
:102588003e510000494500003e000000427f000027
:10259800400000004261000051490000462100004f
:1025a800414500004b31000018140000127f000064
:1025b8001027000045450000453900003c4a00004e
:1025c80049490000300100007109000005030000be
:1025d8003649000049490000360600004949000014
:1025e800291e000000360000360000000000000030
:1025f8005636000000000000000800001422000009
:1026080041140000141400001414000041220000ba
:102618001408000000020000015100000906000033
:1026280032490000794100003e7e0000111100008f
:10263800117e00007f49000049490000363e000035
:1026480041410000412200007f410000412200007a
:102658001c7f000049490000494100007f09000033
:1026680009010000013e0000414100005132000014
:102678007f080000080800007f000000417f00007c
:102688004100000020400000413f0000017f0000a1
:1026980008140000224100007f4000004040000074
:1026a800407f000002040000027f00007f04000059
:1026b800081000007f3e000041410000413e00003c
:1026c8007f09000009090000063e00004151000092
:1026d800215e00007f09000019290000464600001d
:1026e8004949000049310000010100007f01000054
:1026f800013f000040400000403f00001f20000054
:10270800402000001f7f000020180000207f0000ec
:10271800631400000814000063030000047800003c
:102728000403000061510000494500004300000017
:10273800007f000041410000020400000810000072
:1027480020410000417f000000000000040200005a
:10275800010200000440000040400000404000002a
:102768000001000002040000002000005454000092
:10277800547800007f4800004444000038380000c6
:10278800444400004420000038440000444800004d
:102798007f3800005454000054180000087e0000e0
:1027a800090100000208000014540000543c000015
:1027b8007f0800000404000078000000447d000049
:1027c8004000000020400000443d000000000000e0
:1027d8007f10000028440000004100007f400000f6
:1027e800007c000004180000047800007c08000049
:1027f8000404000078380000444400004438000015
:102808007c140000141400000808000014140000d0
:10281800187c00007c080000040400000848000040
:102828005454000054200000043f000044400000bd
:10283800203c000040400000207c00001c200000dc
:10284800402000001c3c000040300000403c0000dc
:102858004428000010280000440c000050500000dc
:10286800503c000044640000544c00004400000048
:102878000836000041000000000000007f00000052
:1028880000000000413600000800000008080000b1
:102898002a1c0000080800001c2a00000808000084
:1028a8002f0f00002000000000f80000f88800004a
:1028b800a0f80000e0000000000000000000000098
:1028c8000000000000000000000000000000000000
:1028d80000000000000000000000000000000000f0
:1028e80000000000000000000000000000000000e0
:1028f80000000000000000000000000000000000d0
:1029080000000000000000000000000000000000bf
:10291800000000000000000000000000000f0000a0
:102928002f00000020a8000000a80000a8f8000060
:10293800a8000000f80000000000000000000000ef
:10294800000000000000000000000000000000007f
:10295800000000000000000000000000000000006f
:10296800000000000000000000000000000000005f
:10297800000000000000000000000000000000004f
:10298800000000000000000000000000000000003f
:102998000000000000f8000000a000000fef000099
:1029a800ff7f000000000000d97f0000b8f9000098
:1029b800627f000074f300009d7e000038ed000087
:1029c8008a7d000007e700002a7c0000e6e000009e
:1029d8007d7a0000d8da000085780000e1d4000094
:1029e8004276000004cf0000b673000046c900001c
:1029f800e3700000a9c30000ca6d000032be0000e9
:102a08006e6a0000e3b80000d0660000c0b30000a2
:102a1800f2620000ccae0000d75e00000aaa0000f7
:102a2800825a00007ea50000f655000029a100008a
:102a3800345100000e9d0000404c00003099000009
:102a48001d47000092950000ce410000369200001c
:102a5800573c00001d8f0000ba3600004a8c000069
:102a6800fc300000be8900001f2b00007b8700009f
:102a780028250000838500001a1f0000d683000067
:102a8800f918000076820000c81200006381000077
:102a98008c0c00009e800000480600002780000083
:102aa8000000000000800000b8f900002780000046
:102ab80074f300009e80000038ed00006381000080
:102ac80007e7000076820000e6e00000d6830000f9
:102ad800d8da000083850000e1d400007c8700007c
:102ae80004cf0000be89000046c900004a8c0000df
:102af800a9c300001d8f000032be000036920000fe
:102b0800e3b8000092950000c0b3000031990000be
:102b1800ccae00000e9d00000aaa000029a100000a
:102b28007ea500007ea5000029a100000aaa0000d9
:102b38000e9d0000ccae000031990000c0b300002b
:102b480092950000e3b800003692000032be000003
:102b58001d8f0000a9c300004a8c000046c9000070
:102b6800be89000004cf00007c870000e1d400008b
:102b780083850000d8da0000d6830000e6e0000074
:102b88007682000007e700006381000038ed00004e
:102b98009e80000074f3000027800000b8f9000050
:102ba8007c7d00007e080000090a00000c0d000072
:102bb8000e10000011120000141500001674000019
:102bc80075760000787900007a7c00007d7e000030
:102bd800080900000a0c00000d0e00007faa000082
:102be8006e800000e69d00007faa00006e7f000056
:102bf8001963000080ab0000220000006869000033
:102c08006a6c00006d6e0000707100007274000044
:102c180075760000787900007a6000006162000033
:102c28006465000066680000696a00006c6d000059
:102c38006e700000717200007faa00006e800000b4
:102c4800960f00007faa00006e7f000069f1000067
:102c580080ab0000220000005455000056580000c8
:102c6800595a00005c5d00005e600000616200006f
:102c780064650000664c00004d4e00005051000095
:102c88005254000055560000585900005a5c000084
:102c98005d5e00007faa00006e800000825c00007c
:102ca8007faa00006e7f00007da4000080ab0000ba
:102cb8002200000040410000424400004546000058
:102cc800484900004a4c00004d4e00005051000099
:102cd80052380000393a00003c3d00003e400000f8
:102ce800414200004445000046480000494a0000af
:102cf8007faa00006e80000065b200007faa000075
:102d08006e7f00009a4e000080ab00002200000099
:102d18002c2d00002e300000313200003435000028
:102d280036380000393a00003c3d00003e240000df
:102d380025260000282900002a2c00002d2e00003e
:102d48003031000032340000353600007fac00001e
:102d5800238000005f1000007fac0000237f00008c
:102d6800a0f0000080a70000b800000000000000ec
:102d7800003f00000ad70000233c000000000000cc
:102d8800003f00000ad70000233c00006f1200003b
:102d9800833b00006f120000833b0000000000002e
:102da8004843000059b10000ae380000cd000000d3
:102db80023870000883c0000c7bb00007b3f000061
:102dc80000fc0000ff460000cdcc0000cc3e000017
:082dd80018720000313f0000f9
:020000040000fa
:102de0001400fa00881f7800cbc2bf000080fb00ef
:102df0004200de00614060000080fb004007980058
:102e0000d2c2bf000080fb004300de0061406000d2
:102e10000080fb00300798003e0090000000e000ba
:102e2000050032000002200020079800f003200077
:102e30001007980004003700800320002007980046
:102e4000d003200010079800beb8a800be98a900c3
:102e50000040eb00504f980079003700de489000aa
:102e600080cbb30000c070001202070000c4b300a2
:102e7000100207005e489000e44f50000d0036003d
:102e80000040eb00704f9800050037000040eb0059
:102e9000170207007e4890000040e800704f98003d
:102ea000fe489000f0c3b30080cf5000f7ff36001b
:102eb000600037005e489000e44f500028003a0060
:102ec0000040eb00704f9800200037007e489000d3
:102ed0008080fb002e009000808f50001100340095
:102ee0007e4890008080fb001e009000808f500084
:102ef0000c003d004e0090000000e00009003a0088
:102f00007e4890000080fb00800040004045290082
:102f100000804000104078000014a000f401070079
:102f2000070037007e4890000080fb0080004000d2
:102f3000404529000080400010407800ec01070067
:102f40007e4890000040e800704f9800fe489000d6
:102f5000f0c3b30080cf5000dcff360035003700ef
:102f60000040eb00704f98002e0037007e48900024
:102f70000080fb008000400000f020000080400046
:102f800010007800604f98006e4890000080fb00b1
:102f90004300de00404f9800ce48900030c0b300a0
:102fa00001405000304f9800ee4890004e4890008d
:102fb0000080fb004300dd0000c05000204f98005f
:102fc000de4890003e48900080cf50000200310063
:102fd0000040eb00c6010700de4890003e4890002c
:102fe00080cf500006003a002e4890008080fb0001
:102ff000c02629000080400010407800bc01070076
:10300000de4890003e48900080cf5000020036001d
:1030100000c0eb00b60107007e4890000040e800c9
:10302000704f9800fe489000f0c3b30080cf50006e
:10303000ceff36005e4890000040e800504f9800f8
:103040005e489000e74f500084ff36003e0090003d
:103050000000e000050032000000eb0020079800af
:10306000f001200010079800040037002000200025
:10307000200798007000200010079800beb8a90033
:10308000be98a8000040eb00504f98007c0037002d
:10309000de48900080cbb30000c0700085010700bf
:1030a00000c4b300830107005e489000e44f500065
:1030b0000d0036000040eb00704f9800050037000f
:1030c0000040eb008a0107007e4890000040e800c5
:1030d000704f9800fe489000f0c3b30080cf5000be
:1030e000f7ff3600630037005e489000e44f500061
:1030f0002a003a000040eb00704f98002200370091
:103100007e4890008080fb002e009000808f500051
:10311000120034007e4890008080fb001e0090006a
:10312000808f50000d003d004e0090000000e00038
:103130000a0032007e4890000080fb000000400042
:103140008000e800404529000080400010407800e1
:103150000014a00066010700080037007e489000b8
:103160000080fb00000040008000e800404529008e
:1031700000804000104078005d0107007e4890000c
:103180000040e800704f9800fe489000f0c3b30084
:1031900080cf5000daff3600360037000040eb00e9
:1031a000704f98002f0037007e4890000080fb0091
:1031b0000004b0008000400000f0200000804000cb
:1031c00010007800604f98006e4890000080fb006f
:1031d0004300de00404f9800ce48900030c0b3005e
:1031e00001405000304f9800ee4890004e4890004b
:1031f0000080fb004300dd0000c05000204f98001d
:10320000de4890003e48900080cf50000200310020
:103210000040eb0036010700de4890003e48900079
:1032200080cf500006003a002e4890008080fb00be
:10323000c026290000804000104078002c010700c3
:10324000de4890003e48900080cf500002003600db
:1032500000c0eb00260107007e4890000040e80017
:10326000704f9800fe489000f0c3b30080cf50002c
:10327000cdff36005e4890000040e800504f9800b7
:103280005e489000e74f500081ff36008041eb0020
:1032900072c0b30001c1b30060c5b300ad00070048
:1032a0008041eb0072c0b30011c1b30010c3b30082
:1032b000a80007008041eb0072c0b30021c1b30039
:1032c000e0c2b300a30007008041eb0072c0b3006e
:1032d00031c1b30090c3b3009e00070021c080003d
:1032e000b0032000808f50001900340038c68000e1
:1032f0006140b9003df50700000f9800110f9800dc
:103300000800e00007003d000200200003782400d0
:103310000e0890009e08900082f40700000f9800ad
:10332000110f98000e0890009e0890003233230081
:1033300033052c00d8f4070002002000032f2400de
:1033400078f40700c0c58800d1c588000b0037009d
:1033500020c08000cf80de0024f50700020020009e
:1033600003f02300ccf40700020020000322240015
:103370006cf40700c0c58800d1c58800c0c58000b6
:10338000d1c5800044f50700e0c588008041eb000e
:1033900062c0b3008040eb0020c5b3006d000700a1
:1033a0008041eb0062c0b30011c0b30030c5b30070
:1033b000680007008041eb0062c0b30021c0b30089
:1033c000c0c4b300630007008041eb0062c0b300db
:1033d00031c0b30000c2b3005e0007008041eb00c3
:1033e00062c0b30041c0b30040c6b300590007003b
:1033f0008041eb0062c0b30051c0b30020c4b300f1
:10340000540007008041eb0062c0b30061c0b3000c
:10341000d0c6b3004f0007008041eb0062c0b3008c
:1034200071c0b30000c2b3004a000700e1c58000cc
:1034300030062000808f500007003600e0c5800075
:103440000002eb0063002000b20020008000eb00cf
:103450000f00070006003700e0c580000002eb0007
:1034600063002000a20020008000eb00080007009d
:103470008041eb0062c0b30081c0b300d0c2b30092
:10348000340007004f0478000080fa0000000600b6
:103490000600fa00000f7800214798003247980094
:1034a000434798005447980023003700be409000df
:1034b0003e4090000040e900304798001e00780030
:1034c000a2002000811f7800110009000200d8002e
:1034d0000001780001007800cf0078000043b000c0
:1034e000de4190004e4190001a0007001e00780057
:1034f000a2002000110009000200d800000f78008f
:103500002e4090000040e900204798002e40900097
:103510000004e00008003a00be4090003e409000e9
:103520000040e90030479800de4190004e41900095
:10353000e0c2b300070007001e00e000dbff3c0014
:103540002e4090000004e000d8ff3d000080fa000b
:10355000000006000600fa00204798003147980056
:1035600042479800534798003e409000f34f500068
:10357000020036000040eb00304798004e409000bb
:1035800067406000404798003e409000e94f50007f
:103590000a003e00beb8a800be98a9003e409000b8
:1035a0000080fb006600b900e440400000c4b300a6
:1035b00000c070003f0007000b003700beb8a90034
:1035c000be98a8003e4090000080fb006600b90055
:1035d0008040780040ccb30080c0400000c4b300fd
:1035e00000c0700033000700ce40900080cbb300d5
:1035f00000c070002f0007000040eb00004f780073
:103600001f0037005e4090000004e0000c003a000c
:103610002e4090008080fb0000fe2f0000804000c4
:103620001e81fb006500b900820040004027290090
:1036300000804000104078002d0007000f00370088
:103640002e4090008080fb0000fe2f000080400094
:103650001e81fb006500b900820040004027290060
:10366000008040001040780000417800024078005f
:103670000080ea008180ea001d0007001e4fe8007c
:1036800040c0b3009e4f1000deff36005e40900049
:103690000004e00003003a000040eb0014000700c3
:1036a0000200370000c0eb00110007000080fa00a4
:1036b000000006000200fa00004f7800be38a900a2
:1036c000be58a900be78a800e18b21009140780087
:1036d00020c1b300a50c07009e40780030c1b300a4
:1036e000a20c0700110007000080fa00000006008d
:1036f0000200fa00004f7800be38a800be58a900aa
:10370000be78a800e18b21009140780020c1b30071
:10371000960c07009e40780030c1b300930c070060
:10372000020007000080fa00000006000000fa0016
:10373000be18a800be78a800e18b21009140780057
:1037400020c1b300890c0700be18a900be78a800ec
:10375000e18b21009140780020c1b300830c070069
:103760000080fa00000006000000fa008a08070046
:10377000beb8a800be98a900f0c3b300cdff0700f3
:1037800000ccb300cbff0700beb8a900be98a800cc
:10379000f0c3b300c7ff070000ccb300c5ff0700ac
:1037a0000080fa00000006003000fa00881f780050
:1037b0000000200080007800404d290000017800c2
:1037c0008101780001e023007000200067f5070008
:1037d00001e0230070002000a0f507000000eb00ce
:1037e000000f7800d9003700f00320009e0f100072
:1037f00024003c009e017800f00320001e005000d1
:10380000c200dd0000e023000080400010017800cd
:10381000f00320001e005000c200dd0000e0230085
:1038200000804000100078000090b900000278008d
:10383000f00320001e0050004200dd008080e80000
:1038400000e023000080400010017800f003200019
:103850001e0050004200dd008080e80000e02300f0
:1038600000804000100078000090b9000000420085
:10387000000178008380410000d0200000804000db
:10388000020878001e007800701798001e0078006b
:103890008000400000d0200000804000100478002c
:1038a0006140b900d1f307005017980061179800e4
:1038b0000800e00007003d0002002000037824001b
:1038c0005e109000ee10900016f30700501798005d
:1038d0006117980042b7840053b784005e109000cf
:1038e000ee1090006cf30700301798004117980015
:1038f00042b7840053b784000000200001f8230081
:1039000007f3070010179800211798001e00780091
:103910008000400000e0200000804000100478009b
:103920006140b900b1f30700700f980001179800cb
:103930000800e00007003d0002002000037824009a
:103940007e0890008e109000f6f20700700f98002d
:10395000011798007e0990008e1190001e109000b3
:10396000ae1090004cf307000001be003e10900026
:10397000ce109000ebf20700c7f3070000017800bb
:10398000fe119000fe1190008380410000e02000b5
:103990000080400002087800f00320009e0f100015
:1039a000690034009e017800f00b20001e005000da
:1039b000c200dd0000e0230000804000100178001c
:1039c000f00b20001e005000c200dd0000e02300cc
:1039d00000804000100078000090b90000027800dc
:1039e000f00b20001e0050004200dd008080e80047
:1039f00000e023000080400010017800f00b200060
:103a00001e0050004200dd008080e80000e023003e
:103a100000804000100078000090b90000004200d3
:103a2000000178008380410000d020000080400029
:103a3000020878001e007800600f98001e007800d1
:103a40008000400000d0200000804000100478007a
:103a50006140b90065f30700400f9800510f9800ce
:103a60000800e00007003d00020020000378240069
:103a70004e089000de089000aaf20700400f980060
:103a8000510f980042b7840053b784004e0890004d
:103a9000de08900000f30700200f9800310f980017
:103aa00042b7840053b784000000200001f82300cf
:103ab0009bf20700000f9800110f98001e0078007d
:103ac0008000400000e020000080400010047800ea
:103ad0006140b90045f3070060079800710798003e
:103ae0000800e00007003d000200200003782400e9
:103af0006e009000fe0090008af2070060079800b8
:103b0000710798006e019000fe0190000e08900071
:103b10009e089000e0f207000001be002e08900011
:103b2000be0890007ff207005bf3070000017800f9
:103b3000ee099000ee0990008380410000e0200033
:103b400000804000020878001e0fe800f007200007
:103b50009e0f100024ff34000000eb0030c68800e8
:103b6000d2c2bf00684060000004e00008003200dc
:103b7000cbc2bf00644060000004e00004003200db
:103b80001004200040c688000006200050c68800af
:103b9000d2c2bf00684060000004e00008003200ac
:103ba000cbc2bf00644060000004e00004003a00a3
:103bb000e001200040c68800d003200050c68800e5
:103bc000d2c2bf00684060000004e00008003a0074
:103bd000cbc2bf00644060000004e000040032007b
:103be0002004200040c688008004200050c68800c1
:103bf000d2c2bf00684060000004e00008003a0044
:103c0000cbc2bf00644060000004e00004003a0042
:103c10006003200040c68800c003200050c6880012
:103c20000000eb00000f78004d0037001e00780008
:103c3000500798001e0078008000400000e020003f
:103c400000804000100478006140b900e7f20700ee
:103c500030079800410798000800e00007003d0089
:103c600002002000037824003e009000ce00900067
:103c70002cf20700300798004107980062b78400d3
:103c800073b784003e009000ce0090001df3070043
:103c90000200200003f8230022f207005bf3070074
:103ca00002002000030424007bf207000200200031
:103cb00003f823001bf20700f7f207000001780069
:103cc000de019000de0190008380410000f02000c2
:103cd00000804000020878001e007800800040004c
:103ce00000f020000080400010007800ff0f50001e
:103cf000060036001e0078008000400000f0200022
:103d000080804000f00120008008780040c68000dc
:103d10009e0f10001100340050c680009e0f10004e
:103d20000e003d001e0078008000400000e02000f2
:103d3000008040009000780030c68000808f5000e6
:103d4000060036001e0078008000400000e02000e1
:103d5000008040001000780030c688001e0fe80088
:103d6000f00720009e0f1000b0ff340038c680001e
:103d70006140b9009df207001007980021079800e4
:103d80000800e00007003d00020020000378240046
:103d90001e009000ae009000e2f1070010079800ae
:103da000210798001e009000ae00900017f3070056
:103db00062b7840073b78400d2f207006af207008a
:103dc00030c68800e17b8000007c800000804000dd
:103dd0000000d100f07b88004f0478000080fa00da
:103de000000006000000fa00ca82a900ca82a800ea
:103df0000001eb008000eb00000320003806070004
:103e0000000000001200200011002000000320002c
:103e10003306070000000000120020008000eb00c5
:103e2000000320002e060700820020001100200061
:103e3000000320002a0607001200200021002000b5
:103e400000032000260607000001eb008000eb00c5
:103e50000003200022060700d2042000b101200048
:103e6000000320001e060700320020004100200051
:103e7000000320001a0607008200200061002000d5
:103e800000032000160607007200200071002000c9
:103e90000003200012060700020820008100200015
:103ea000000320000e060700020a2000e1012000a6
:103eb000000320000a06070012092000510020001c
:103ec000000320000606070022002000d100200089
:103ed00000032000020607000001eb00e1002000c3
:103ee00000032000fe050700020820004101200019
:103ef00000032000fa05070082082000b10020001e
:103f000000032000f605070022082000c100200061
:103f100000032000f2050700820820002101200094
:103f200000032000ee050700820820003101200078
:103f300000032000ea050700820020008000eb005b
:103f400000032000e60507000000000092072000a3
:103f50008101200000032000e105070000000000af
:103f6000320a20009101200000032000dc05070038
:103f700000000000d2002000a1012000000320006a
:103f8000d70507000000000062082000c1012000e2
:103f900000032000d205070000000000c205200039
:103fa000d101200000032000cd0507000000000023
:103fb000320f2000e101200000032000c8050700a7
:103fc0000000000032072000010220000003200052
:103fd000c305070000000000620420001102200059
:103fe00000032000be05070000000000b201200011
:103ff0002102200000032000b90507000000000096
:10400000920020008000eb0000032000b4050700b0
:1040100000000000920720000102200000032000a1
:10402000af05070000000000320a20001102200046
:1040300000032000aa05070000000000d2002000b5
:104040002102200000032000a50507000000000059
:10405000620820004102200000032000a0050700a4
:1040600000000000c20520005102200000032000d3
:104070009b05070000000000320f200061022000b5
:104080000003200096050700000000003207200012
:1040900081022000000320009105070000000000bd
:1040a0006204200091022000000320008c0507001c
:1040b00000000000b2012000a10220000003200047
:1040c00087050700000000000001eb008000eb0006
:1040d00000032000820507000000000022002000ed
:1040e000d1032000000320007d0507000000000030
:1040f000ab0b07006c0b07002d0b0700ee0a070047
:1041000055090700120020008000eb00000320008a
:10411000730507000000000042062000d1032000c4
:10412000000320006e050700000000000001eb0006
:104130003100200000032000690507000000000096
:104140000001eb004100200000032000640507008f
:1041500000000000120020008000eb00000320009f
:104160005f0507000000000082002000c100200061
:10417000000320005a050700000000008200200014
:10418000d1002000000320005505070000000000ba
:1041900082002000e10020000003200050050700fd
:1041a00082002000f1002000000320004c050700e1
:1041b0000001eb008000eb00000320004805070031
:1041c0000000000022002000010420000003200065
:1041d00043050700000000000001eb00110420006f
:1041e000000320003e05070000000000420d2000f3
:1041f000f103200000032000390507000000000043
:10420000120020008000eb000003200034050700ae
:1042100000000000a2002000010120000003200097
:104220002f05070000000000a2002000110120005f
:10423000000320002a050700000000000001eb0039
:1042400021012000000320002505070000000000d8
:104250000001eb00310120000003200020050700d1
:1042600000000000c2032000910020000003200095
:104270001b050700120020008000eb000003200057
:104280001705070000000000020320004103200082
:1042900000032000120507000000000002032000b8
:1042a00071032000000320000d050700000000003e
:1042b00032002000610320000003200008050700f1
:1042c00000000000320020009103200000032000c5
:1042d000030507000000000082022000b103200057
:1042e00000032000fe0407000000000082022000fe
:1042f000c103200000032000f904070000000000b3
:104300000001eb008000eb0000032000f404070034
:1043100000000000020c2000110520000003200016
:10432000ef040700000000000001eb002105200061
:1043300000032000ea040700000000000080fa00eb
:10434000000006000000fa00c1c28000f00f20004b
:104350000080600090c5880090c58000b0f8b7006c
:10436000018b2100914078000000eb000005070060
:10437000c1c2800000f02f0000806000a0c588004e
:10438000a0c580004880de00b0f8b700018b210096
:104390009140780010002000f5040700d1c2800091
:1043a000f00f20000080600090c5880090c580005c
:1043b000b0f8b700018b2100914078002000200068
:1043c000eb040700d1c2800000f02f0000806000e5
:1043d000a0c58800a0c580004880de00b0f8b70006
:1043e000018b21009140780030002000e00407009c
:1043f000e1c28000f00f20000080600090c58800be
:1044000090c58000b0f8b700018b21009140780082
:1044100040002000d6040700e1c2800000f02f0019
:1044200000806000a0c58800a0c580004880de0034
:10443000b0f8b700018b21009140780050002000b7
:10444000cb040700f1c28000f00f20000080600064
:1044500090c5880090c58000b0f8b700018b21009e
:104460009140780060002000c1040700f1c2800084
:1044700000f02f0000806000a0c58800a0c580006b
:104480004880de00b0f8b700018b21009140780031
:1044900070002000b604070021c58000f00f200046
:1044a0000080600090c5880090c58000b0f8b7001b
:1044b000018b21009140780080002000ac040700af
:1044c00021c5800000f02f0000806000a0c588009a
:1044d000a0c580004880de00b0f8b700018b210045
:1044e0009140780090002000a104070031c58000b1
:1044f000f00f20000080600090c5880090c580000b
:10450000b0f8b700018b210091407800a000200096
:104510009704070031c5800000f02f000080600084
:10452000a0c58800a0c580004880de00b0f8b700b4
:10453000018b210091407800b00020008c0407001e
:1045400041c58000f00f20000080600090c5880009
:1045500090c58000b0f8b700018b21009140780031
:10456000c00020008204070041c5800000f02f0039
:1045700000806000a0c58800a0c580004880de00e3
:10458000b0f8b700018b210091407800d0002000e6
:104590007704070001c08000f00f20000080600059
:1045a00090c5880090c58000b0f8b700018b21004d
:1045b00091407800e00020006d04070001c08000f9
:1045c00000f02f0000806000a0c58800a0c580001a
:1045d0004880de00b0f8b700018b210091407800e0
:1045e000f0002000620407000080fa0000000600ce
:1045f0000000fa000000eb0087040700b6f8b700df
:10460000b6d8bf008000fb00f00f200000806000e3
:1046100090c58800100020007f040700b6f8b7009e
:10462000b6d8bf000000fb004800dd00a0c5880030
:10463000a1c5800090c5800000807000c0c28800c5
:1046400000000000000000002000200072040700ad
:10465000b6f8b700b6d8bf008000fb00f00f20000e
:104660000080600090c58800300020006a040700c8
:10467000b6f8b700b6d8bf000000fb004800dd0068
:10468000a0c58800a1c5800090c580000080700092
:10469000d0c28800000000000000000040002000a0
:1046a0005d040700b6f8b700b6d8bf008000fb0075
:1046b000f00f20000080600090c5880050002000ae
:1046c00055040700b6f8b700b6d8bf000000fb00dd
:1046d0004800dd00a0c58800a1c5800090c580000d
:1046e00000807000e0c288000000000000000000b0
:1046f0006000200048040700b6f8b700b6d8bf0035
:104700008000fb00f00f20000080600090c5880052
:104710007000200040040700b6f8b700b6d8bf000c
:104720000000fb004800dd00a0c58800a1c5800096
:1047300090c5800000807000f0c28800000000007a
:10474000000000008000200033040700b6f8b70026
:10475000b6d8bf008000fb00f00f20000080600092
:1047600090c58800900020002b040700b6f8b70021
:10477000b6d8bf000000fb004800dd00a0c58800df
:10478000a1c5800090c580000080700020c5880011
:104790000000000000000000a00020001e04070030
:1047a000b6f8b700b6d8bf008000fb00f00f2000bd
:1047b0000080600090c58800b0002000160407004b
:1047c000b6f8b700b6d8bf000000fb004800dd0017
:1047d000a0c58800a1c5800090c580000080700041
:1047e00030c588000000000000000000c00020006c
:1047f00009040700b6f8b700b6d8bf008000fb0078
:10480000f00f20000080600090c58800d0002000dc
:1048100001040700b6f8b700b6d8bf000000fb00df
:104820004800dd00a0c58800a1c5800090c58000bb
:104830000080700040c588000000000000000000fb
:10484000e0002000f4030700b6f8b700b6d8bf00b8
:104850008000fb00f00f20000080600090c5880001
:10486000f0002000ec030700b6f8b700b6d8bf0090
:104870000000fb004800dd00a0c58800a1c5800045
:1048800090c580000080700000c08800000000001b
:10489000000000000080fa00000006000000fa009e
:1048a000889fbe0050c48000cf80de00cfef07009d
:1048b0000001be0000002000a137240011f0070015
:1048c000a9f0070002002000031a240072ef07007d
:1048d00020c1880031c1880020c1800031c1800022
:1048e0006011b800a4f007000000e00001003c00e7
:1048f0001400370080c1800091c1800022c1800077
:1049000033c1800064ef07000004be0082c1800054
:1049100093c180000000200001f8230000ef070091
:1049200062c1800073c180005bef07000001be0020
:104930000800be00fbee070040c1880051c188009e
:1049400013003700a0c18000b1c1800022c18000e7
:1049500033c1800050ef07000004be00a2c18000f8
:10496000b3c180000000200001f82300ecee070036
:1049700062c1800073c1800047ef07000001be00e4
:104980000800be00e7ee070040c1880051c1880062
:1049900040c1800051c1800073ef07000001be00dc
:1049a000f0ff2f00f1ff2700800f5100818f590089
:1049b00003003a006000b80040c1880051c188007f
:1049c00040c1800051c1800060c1880071c1880071
:1049d00040c1800051c1800063ef07008000780073
:1049e00020c080000080400020c0880020c08000df
:1049f0000000e00002003d000000eb0020c0880045
:104a000021c08000c0032000808f500002003400cd
:104a1000c003200020c0880021c0800030c080007a
:104a2000808f50000400320020c08000d3040700b3
:104a300020c0800030c0880090b68400a1b68400f9
:104a40000004be0000c58000cf80de0067ef0700d5
:104a50000001be000800be00aaef070042f00700f8
:104a600002002000032024000bef070000c1880093
:104a700011c1880000c58000cf80de005bef070019
:104a800092b68400a3b684003bf007000000e0006b
:104a900001003d001100370080c0800091c08000ff
:104aa00002c1800013c18000fbee07000004be00bd
:104ab000a0c08000b1c08000e2c08000f3c08000d0
:104ac000f5ee07000001be000800be0095ee0700ed
:104ad000c0c08800d1c088001000370040c08000ee
:104ae00051c0800002c1800013c18000eaee0700bf
:104af0000004be0060c0800071c08000e2c0800081
:104b0000f3c08000e4ee07000001be000800be0014
:104b100084ee0700c0c08800d1c08800e0c08000db
:104b2000f1c0800010ef07000001be00f0ff2f0071
:104b3000f1ff2700800f5100818f590003003a00d8
:104b40006000b800e0c08800f1c08800c0c08000ec
:104b5000d1c0800004ef07000001be00f0ff2f006d
:104b6000f1ff2700800f5100818f590003003a00a8
:104b70006000b800c0c08800d1c08800c0c08000fc
:104b8000d1c08000e0c08800f1c08800c0c08000b3
:104b9000d1c08000f4ee07008000780000c08000e3
:104ba00000804000c0c18800c1c18000d0c1800029
:104bb000808f500004003200c0c180008d040700c7
:104bc000c0c18000d0c188004f04be000080fa0040
:104bd000000006000000fa0090042100e19223008a
:104be00080c1880091c18800b0b68400c1b684003d
:104bf0000200200003302400a7ee0700d2b5840095
:104c0000e3b584003fef070080c1880091c18800b0
:104c1000b0b68400c1b68400020020000330240036
:104c20009dee0700f2b5840003b6840035ef07005f
:104c3000a0c18800b1c18800b0b68400c1b68400ac
:104c4000020020000330240093ee070012b6840017
:104c500023b684002bef070040c0880051c08800b5
:104c6000b0b68400c1b684000200200003302400e6
:104c700089ee070032b6840043b6840021ef0700b6
:104c800080c0880091c0880042c0800053c080006e
:104c90000000200001f8230021ee070060c088001a
:104ca00071c0880082c0800093c080000000200096
:104cb00001f823001aee0700a0c08800b1c08800e8
:104cc00050b6840061b68400b2b68400c3b68400d6
:104cd0000cef0700a4ee0700e0c4880070b6840063
:104ce00081b68400b2b68400c3b6840005ef070025
:104cf0009dee0700d0c488000000eb0000c58800ce
:104d00000000eb0010c588006000b800c0c088003b
:104d1000d1c088006000b800e0c08800f1c0880001
:104d20000000eb0050c488000000eb0060c4880065
:104d30000000eb0010c08800c003200020c08800e5
:104d400020c0800030c088000080fa00000006000b
:104d50000200fa00cac2bf00684060000004e00020
:104d60000f003a00cae2a900d2c2bf007040600042
:104d70000004e00005003a002000200070c5880013
:104d80000000eb0050c588000c0037000000eb006d
:104d900070c588001000200050c58800070037004b
:104da0001000200070c58800cae2a800000820009a
:104db000c0c388000000eb0010c68800cbc2bf0053
:104dc000684060000004e0000d0032001200200086
:104dd0008000eb00000320004102070000000000fb
:104de0000204200031032000000320003c020700e1
:104df0000000000020c5800070c288000c00370051
:104e0000120020008000eb000003200034020700a5
:104e1000000000000001eb0031032000000320002f
:104e20002f0207000000000030c5800070c288001b
:104e300070c58000000f78001e007800e10f500060
:104e40002f0032001e007800e20f500056003200a2
:104e50001e0078000000e000010032006d00370005
:104e6000000420009b030700120020008000eb00dc
:104e7000000320001a020700000000000001eb0000
:104e8000410320000003200015020700000000007d
:104e90000001eb0071032000000320001002070056
:104ea000000000000000eb00d20307000000eb0050
:104eb000f3030700c00020009b030700120020003e
:104ec0008000eb0000032000050207000000000046
:104ed000c200200041032000000320000002070060
:104ee0000000000070c28000a4030700c0c2800060
:104ef00030608800d0c280005060880045003700d4
:104f0000000420007303070000042000860307004c
:104f1000120020008000eb0000032000f0010700d9
:104f2000000000000001eb0041032000000320000e
:104f3000eb010700000000000001eb0071032000fe
:104f400000032000e601070000000000020320002b
:104f50004103200000032000e101070000000000e1
:104f6000020320007103200000032000dc01070081
:104f70000000000000c080009e03070020c08000e9
:104f80007e030700c0fe2f00bd0307006000200065
:104f900050030700e0c2800030608800f0c280004b
:104fa000506088001b003700000420004903070000
:104fb000120020008000eb0000032000c801070061
:104fc000000000000001eb0041032000000320006e
:104fd000c3010700000000000001eb007103200086
:104fe00000032000be0107000000000040c5800053
:104ff00080030700800120004b0307000000eb0046
:1050000034030700c0c2800030608800d0c2800036
:1050100050608800cbc2bf00644060000004e00024
:10502000030032000080eb0060c5880002003700fa
:105030001000200060c58800cac2bf006440600044
:105040000004e0001a003a00ab00070000c3800033
:10505000e30f50000300320000c38000e70f500050
:1050600012003a00b0cc2600c0c288000000eb005d
:10507000d0c28800b0cc2600e0c288000000eb005f
:10508000f0c288000000eb0020c588000000eb00a3
:1050900030c588000000eb0040c588000000eb0030
:1050a00000c08800a7fc070001003700a5fc07002e
:1050b000cac2bf000080fb004500de006140600006
:1050c00061416000212d200091407800e0cfb300c5
:1050d00000c0600002407000d2e2b700cac2bf0048
:1050e0000080fb004600de0061406000614060001f
:1050f00000414000212d200091407800d0cfb30026
:1051000000c0600002407000d2e2b700cbc2bf0016
:105110000080fb004200de006140600061406000f2
:105120004201dd00212d200091407800b0cfb30076
:1051300000c0600002407000d2e2b700cbc2bf00e6
:105140000080fb004300de0061406000c700dd001e
:10515000c2c2bf000074a10001407000c2e2b700eb
:10516000cac2bf000080fb004300de006140600057
:10517000614060004201dd00312c20009140780048
:10518000b0cfb30000c0600002407000c3e2b700bf
:105190000080fa00000006000000fa003000200045
:1051a00010c288002000200020c288001116800054
:1051b00010c2800000806000e0c188003000200044
:1051c00010c38800b0fe270030c28800b05225000e
:1051d00040c288008038210050c2880080c72e005d
:1051e00060c288000005200080c288000000eb003b
:1051f00090c2880000032000a0c2880040ff2f005a
:10520000b0c288000080fa00000006000000fa002a
:1052100000c28000e20f50000a003a0071c2800014
:1052200090c28000808f50000f00340070c2800058
:105230000000e90070c2880070c28000cf02070041
:105240000900370071c2800080c28000808f50004a
:1052500005003d0070c280000000e80070c28800b8
:1052600070c28000c5020700cbc2bf00684060006a
:105270000004e0000300320070c2800020c58800f6
:105280000200370070c2800030c588000080fa003c
:10529000000006000000fa0000c28000e20f50008b
:1052a0000a003a0041c58000b0c28000808f5000e3
:1052b0000f00340040c580000000e90040c58800b0
:1052c00040c58000cb0207000900370041c58000bf
:1052d000a0c28000808f500005003d0040c58000c6
:1052e0000000e80040c5880040c58000c1020700fa
:1052f0000080fa00000006000000fa00501680004e
:1053000000c3880000c380004580de0000c3880021
:1053100001c3800010c380000080600000c38800cb
:1053200070c58000e10f50000300320000c3800010
:105330006400400000c388000080fa0000000600fe
:105340000200fa00e0c1800000004000e0c18800d7
:10535000e1c18000f0c180000080680000c28800c8
:1053600001c2800020c280000080600000c288006e
:10537000e1ff070000c38000000f78001e007800e6
:10538000e30f50008e0032001e007800e30f500043
:105390000a003c001e007800e10f50002a00320095
:1053a0001e007800e10f50003d003c001e00780018
:1053b0000000e0000b003200810037001e00780082
:1053c000e50f5000530032001e007800e50f50003a
:1053d000490035001e007800e60f500063003200df
:1053e0007700370000c28000e20f500003003a004f
:1053f000c0ff2f0010c088000200370040002000ce
:1054000010c0880001c0800010c0800000804000f3
:1054100000c0880001c0800000032000808f500081
:10542000020034000003200000c0880001c080009a
:1054300010f82f00808f500061003d0010f82f0001
:1054400000c088005e00370000c28000e20f5000fc
:1054500009003a00e1c2800040c28000808f500005
:105460000c003400e0c28000c1f92f0001004000b0
:10547000e0c2880007003700e1c2800030c280002f
:10548000808f500003003d00e0c280004006b00065
:10549000e0c28800e0c28000306088004800370029
:1054a00000c28000e20f500009003a00f1c2800003
:1054b00060c28000808f50000c003400f0c2800079
:1054c000c1f92f0001004000f0c28800070037003a
:1054d000f1c2800050c28000808f500003003d0068
:1054e000f0c280004006b000f0c28800f0c2800028
:1054f000506088003200370050c580000000e00096
:1055000002003a0063ff07002d0037003fff07004d
:105510002b00370000c28000e20f500009003a0063
:10552000c1c2800040c28000808f50000c00340057
:10553000c0c28000c1f92f0001004000c0c2880035
:1055400007003700c1c2800030c28000808f500049
:1055500003003d00c0c280004006b000c0c2880009
:10556000c0c28000306088001500370000c2800093
:10557000e20f500009003a00d1c2800060c28000f2
:10558000808f50000c003400d0c28000c1f92f0081
:1055900001004000d0c2880007003700d1c280005f
:1055a00050c28000808f500003003d00d0c28000b8
:1055b0004006b000d0c28800d0c280005060880091
:1055c000f0c18000e0c188000080fa000000060001
:1055d0000000fa000000eb00001088000000eb0063
:1055e000101088000000eb00501088000000eb0055
:1055f0006010880000042000201088000602a90026
:10560000000000000622a900000000000642a900d8
:10561000000000000662a900000000000682a90048
:105620000000000006a2a9000000000006c2a900b8
:105630000000000006e2a900000000000702a90027
:10564000000000000722a900000000000742a90096
:10565000000000000762a900000000000782a90006
:105660000000000007a2a9000000000007e2a80057
:10567000000000000802a900000000000822a900a4
:10568000000000000842a900000000000862a90014
:10569000000000000882a9000000000008a2a90084
:1056a0000000000008c2a9000000000008e2a900f4
:1056b000000000000902a900000000000922a90062
:1056c000000000000942a9000000000009c2a90072
:1056d0000000000009e2a9000080fa0000000600b6
:1056e0000400fa00004f7800114798002247980004
:1056f0000602a800301080007f0060000000e0007b
:10570000fcff3a001e80fb001010880009c2bf0099
:105710000044b2000004e000fcff3a001e4090008c
:105720000080fb001010880009c2bf000044b200d6
:105730000004e000fcff3a002e4090000080fb00d7
:105740001010880009c2bf000044b2000004e0004d
:10575000fcff3a000642a80006c2bf006440600099
:105760000004e000fcff3a000080fa0000000600a0
:105770000400fa00000f7800214798000602a800f4
:10578000301080007f0060000000e000fcff3a0065
:10579000000a20001010880009c2bf000044b200b7
:1057a0000004e000fcff3a001e0078004880de00a4
:1057b0001010880009c2bf000044b2000004e000dd
:1057c000fcff3a001e0078001010880009c2bf00dc
:1057d0000044b2000004e000fcff3a002e409000bc
:1057e0000000fb001010880009c2bf000044b20096
:1057f0000004e000fcff3a000642a80006c2bf0019
:10580000644060000004e000fcff3a00570007001d
:105810000080fa00000006000400fa00100798005b
:105820000602a80006c2bf00614060000004e0005c
:10583000fcff3a00000a20001010880009c2bf00d7
:105840000044b2000004e000fcff3a001e0090009b
:105850004880de001010880009c2bf000044b2007a
:105860000004e000fcff3a001e00900010108800c9
:1058700009c2bf000044b2000004e000fcff3a008f
:105880000622a80006c2bf00624060000004e000db
:10589000fcff3a00100a20001010880009c2bf0067
:1058a0000044b2000004e000fcff3a0009c2bf005f
:1058b00001c8b300014060000004e000fbff3a00b3
:1058c0000662a80006c2bf00684060000004e00055
:1058d000fcff3a0000108000004f780006a2a800ec
:1058e0000682a80006c2bf00704060000004e0000d
:1058f000fcff3a000642a80006c2bf0064406000f8
:105900000004e000fcff3a001e00fb000080fa00eb
:10591000000006000200fa000000eb00000f780013
:1059200002003700000000001e0fe8007000200099
:105930009e0f1000fbff34000080fa0000000600fc
:105940000200fa000000eb00000f780002003700b0
:10595000000000001e0fe800f0f920009e0f10006c
:10596000fbff34000080fa00000006000200fa008d
:105970000000eb00000f780002003700f0ff070086
:105980001e0fe800100320009e0f1000fbff3400e4
:105990000080fa00000006000200fa000000eb00a0
:1059a000000f780002003700e5ff07001e0fe80037
:1059b000900f20009e0f1000fbff34000080fa00c3
:1059c000000006003600f800809fbe00829fbe00e7
:1059d000849fbe00869fbe00889fbe000200fa0022
:1059e0008b80a90070c58000000f78001e01780030
:1059f000e10f5100150032001e007800e20f500048
:105a0000460032001e0178000200e0000100320072
:105a1000a80037008014800020608800206080008b
:105a2000906088009014800000c488006a0307001a
:105a300040608000c0148800b160800060c58000b4
:105a40000088b900d01488009a00370090148000b4
:105a5000e0c3880080148000f0c38800c0c38000c9
:105a6000e2c3800080004000000021000080400070
:105a700002087800c0c38000f2c3800080004000ac
:105a8000002021000080400002087800c0c3800090
:105a90000000e800c0c38800c1c3800000082000e7
:105aa000808f500005003a0010002000d0c388000d
:105ab0000000eb00b0c388009460a800c1c3800060
:105ac00000102000808f500007003a000000eb001b
:105ad000c0c3880010002000d0c388000008200048
:105ae000b0c388009460a800c0c38000800040005c
:105af000004021000080400010007800c0148800a1
:105b0000c0c3800080004000006021000080400091
:105b100010007800d01488006600370021c3800090
:105b2000d0b684000080400020c3880020c38000dd
:105b300002002100110009000200d8008000fd00d1
:105b400020c38800d2c2bf000042b2000004e000bf
:105b5000040032006000b80010c4880021c488002e
:105b60000400370020b7840031b7840010c48800d7
:105b700021c4880010c4800021c4800052c380006a
:105b800063c3800066ea0700e2b68400f3b68400cf
:105b9000c1ea07000004be0000b7840011b784000a
:105ba00052c3800063c38000bbea07000001be004f
:105bb0000800be005bea070030c3880041c38800cc
:105bc00030c3800041c3800092c38000a3c3800023
:105bd00053ea0700e2b68400f3b68400aeea070099
:105be0000004be0000b7840011b7840092c3800097
:105bf000a3c38000a8ea07000001be000800be00a1
:105c000048ea070070c3880081c3880030c3800061
:105c100041c3800050c3880061c3880090c38000e6
:105c2000a1c3800090c38800a1c3880080148000b5
:105c300000c488009014800000c4880070c38000f5
:105c400081c38000c8ea07000004be0020c38000b2
:105c5000d90307006103b9008800780006007800c6
:105c6000000ab80007c0b900050178000001410032
:105c700009b0b90000014100820278004129dd002d
:105c80004f20de0000007100cfa8de0020608800f9
:105c90002060800090608800cf0207004060800094
:105ca000c0148800b160800060c580000088b90021
:105cb000d01488000080fa004f04be004f03be00dd
:105cc0004f02be004f01be004f00be003600f9007b
:105cd000004006000200fa00000f780012c0b30076
:105ce0008040eb0000c3b3007dfe07000000000011
:105cf0001e0078000041780001c1b30000c3b3006a
:105d000077fe0700000000001e00780000417800c8
:105d100011c1b30000c3b30071fe07000000000012
:105d20000080fa00000006000200fa00000f780070
:105d300012c0b3008040eb0000c3b30068fe070050
:105d4000000000001e0078000041780021c1b3006f
:105d500000c3b30062fe0700000000001e007800d0
:105d60000041780031c1b30000c3b3005cfe0700fe
:105d7000000000000080fa00000006000200fa00a7
:105d8000000f78001e00e00002003d000000eb0064
:105d9000000f7800f00520009e0f10000200340074
:105da000f0052000000f780012c0b3008040eb0027
:105db00000c3b3004afe0700000000001e00780088
:105dc00000417800b1c3b30000c3b30044fe070034
:105dd000000000001e00780000417800c1c3b3003d
:105de00000c3b3003efe0700000000000080fa0080
:105df000000006000200fa00000f780000032000f7
:105e00009e0f10000200340000032000000f7800f5
:105e100010f82f009e0f100002003d0010f82f0018
:105e2000000f78001e00e00002003d00001020007e
:105e30001e0f40000041eb008040eb0000c3b300a8
:105e400027fe0700000000001e00780000417800d7
:105e500011c4b30000c3b30021fe0700000000001e
:105e60001e0078000041780021c4b30000c3b300d5
:105e70001bfe0700000000000080fa000000060082
:105e80000200fa00000f7800800220009e0f100030
:105e90000200340080022000000f780080fe2f00f6
:105ea0009e0f100002003d0080fe2f00000f7800c2
:105eb0001e00e00002003d00f00720001e0f400021
:105ec0000041eb008040eb0000c3b30004fe07007c
:105ed000000000001e0078000041780031c5b300ca
:105ee00000c3b300fefd0700000000001e007800a4
:105ef0000041780041c5b30000c3b300f8fd0700be
:105f0000000000000080fa00000006000a00fa000d
:105f10000000eb002007980081003700b1c380002b
:105f20002e00900000804000800040000000210012
:105f30000080400090007800110798001e0090003b
:105f400020608800b1c380002e00900000804000d7
:105f5000800040000020210000804000100f7800e9
:105f60009e00780091608800a0c4800000618800d5
:105f700019020700b160800060c580000088b90088
:105f8000b060880041608000b06080000080400008
:105f9000a0c48800d2c2bf00684060000004e000d6
:105fa00003003200a0c4800080c4880002003700d3
:105fb0001061800080c48800b1c380002e00900072
:105fc0000080400082c4800080004000004021002a
:105fd0000080400002087800b1c380002e009000cd
:105fe0000080400082c480008000400000602100ea
:105ff000008040000208780040c480000000e000fb
:1060000018003a0030c4800062608000c200dd00e9
:1060100000e02300008040000208780030c48000c7
:10602000d26080004200dd008080e80000e02300b4
:10603000008040000208780030c480000000e800c2
:1060400030c4880031c4800000082000808f5000d8
:1060500004003a000000eb0030c48800100020006b
:1060600040c488001e00900040079800ce009000b9
:106070000100e00003003d004e0090000000ea0037
:1060800040079800ce00900071c4880071c4800061
:1060900060c4800000805000e2c48000110009004c
:1060a0000200d8008000780060c4800000804000ba
:1060b00050c4880050c4800060c4880080c4800040
:1060c000300798003e0090000000e00003003d0013
:1060d000be0090008100ea00310798003e00900069
:1060e000f0c48800f1c4800010c58000008050001a
:1060f000d2c48000110009000200d800800078009e
:1061000010c580000080400000c5880000c58000e8
:1061100010c588002e0090000000e80020079800bd
:10612000ae009000f0072000808f50007bff34000d
:106130000080fa00000006000200fa0000082000bb
:1061400010308a00008020001060880010608000fd
:10615000f00fb0000060880000302400e00fb000b5
:1061600000308a000008200030308a0000902000b3
:106170008060880080608000f00fb0007060880050
:1061800000402400e00fb00020308a000000eb0047
:10619000000f7800210037001e00780080004000ca
:1061a00000802000808040000000eb008008780024
:1061b0001e0178001e0078008000400060f6280074
:1061c00000804000900178008200410000302400ef
:1061d00000804000030878001e0078008000400026
:1061e00000902000808040000000eb0080087800d4
:1061f0001e0178001e007800800040006006290023
:10620000008040009001780082004100004024009e
:1062100000804000030878001e0fe800f00720000f
:106220009e0f1000dcff3400f007200050308a0081
:1062300000a02000f0608800f0608000d00fb00067
:10624000e060880000502400c00fb00040308a0099
:106250000000eb00000f7800110037001e007800ee
:106260008000400000a02000808040000000eb0083
:10627000800878001e0178001e0078008000400031
:1062800060162900008040009001780082004100e3
:106290000050240000804000030878001e0fe80032
:1062a000e00720009e0f1000ecff3400b0cc260069
:1062b000a06088000080fa00000006000200fa00da
:1062c0000000eb00000f78000d0037001e00780082
:1062d0008000400000a02000808040000000eb0013
:1062e000800878001e0078008000400000502400e4
:1062f000808040000000eb00800878001e0fe8005e
:10630000e00720009e0f1000f0ff34000080fa002c
:10631000000006000000fa00313a800000e02f0083
:10632000008060009001b300303a88000000000057
:1063300044c7bf00f043b20044e7b70000000000cc
:10634000417420009140780000ceb30000c060008e
:1063500044e7b70000000000320020008107200061
:10636000a00920003374200081497800804978001a
:10637000824978001200200061042000700520008e
:106380002374200081497800804978008249780090
:1063900043c7bf0002c7b3008240600000c3b30020
:1063a00080cf5000faff3a000000000088fc070090
:1063b000000000004600070000000000b6010700d2
:1063c000000000006001070000000000e6f4070084
:1063d000000000005e0307000000000081f60700d7
:1063e00000000000a60307000000000052ff0700a5
:1063f000000000007ef807000000000066fb0700b8
:1064000000000000f3f9070000000000b4030700db
:10641000000000004efa070000000000000000002d
:1064200000082000c0c388000000eb0010c68800f0
:106430000000370040c48000e10f500008003a001f
:1064400010c68000e20f500005003a00d6f40700a5
:106450000000eb0040c488001000200000c6880047
:1064600000c68000e10f500006003a0010c6800010
:10647000e40f500003003a0059f207000000eb005f
:1064800000c6880060c68000e10f500003003a009b
:106490002ffa07000000eb0060c68800111680008c
:1064a00010c2800000806000f0c18800f1c180004f
:1064b000e0c180000080680020c6880020c68000ff
:1064c0000000e000dbff32009dfb0700d9ff370032
:1064d0000000fa002d23a800000000002d43a800b2
:1064e000000000002d63a800000000002d83a8001c
:1064f000000000002c03a800000000002c23a800ce
:10650000000000002c83a800000000002ca3a800bd
:10651000000000002cc3a800000000002ce3a8002d
:10652000000000002d03a80000000000c882a900a0
:1065300000000000c8e2a90000000000c982a90014
:1065400000000000d002a90000000000d022a90035
:1065500000000000d042a90000000000c142a900d4
:1065600000000000c0e2a90000000000c16c200093
:106570009140780000ceb30000c06000d040b3006e
:10658000cce6b70000000000116b200091407800bd
:1065900000ceb30000c06000d040b300b1e6b70049
:1065a00000000000216b20009140780000ceb30075
:1065b00000c06000f040b300b2e6b7000000000089
:1065c000016b20009140780000ceb30000c0600055
:1065d000e040b300b0e6b700000000006840a8004b
:1065e000000000006860a8000000000068c0a8006b
:1065f0000000000068e0a8000000000069e0a800ba
:10660000000000006a00a800000000006b00a80065
:10661000000000006b20a800000000006b40a800f4
:10662000000000006b60a800000000006b80a80064
:106630000000000060c0a80060e0a80061e0a800c1
:106640006200a8006360a8006300a8006320a8009f
:106650000080fa00000006003000fa000e80e8001a
:10666000215f29000e00090031587800f000b100c8
:1066700071004700315e29000e0009003158780092
:10668000f000b100000220000e004000415d290032
:106690000e00090031587800f000b1000000eb0056
:1066a000000f780082c0b3008040eb0000c3b3004d
:1066b0000bfc0700000000000a0037009e00780075
:1066c0000e80e800614178009e007800710047006c
:1066d000e140780000c3b30001fc070000000000a7
:1066e0001e0fe800800020009e0f1000f3ff340012
:1066f00092c0b3008040eb0000c3b300f8fb07007a
:10670000000000000a0037009e0078000e80e800bc
:10671000614178009e00780071004700e1407800f8
:1067200000c3b300eefb0700000000001e0fe800ee
:10673000e10020009e8f1000f3ff34000000eb000a
:10674000000f78000b0037009e0078000e80e800f4
:10675000614178009e007800000220000e00400099
:10676000e140780000c3b300ddfb0700000000003b
:106770001e0fe800200020009e0f1000f2ff3400e2
:10678000a2c0b3008040eb0000c3b300d4fb0700fd
:10679000000000000b0037009e0078000e80e8002b
:1067a000614178009e007800000220000e00400049
:1067b000e140780000c3b300c9fb070000000000ff
:1067c0001e0fe800e10020009e8f1000f2ff340051
:1067d0000080fa00000006004600f8004800f800bb
:1067e0004a00f8004400f8003400f8003600f800d1
:1067f000851f7800861f7800881f78008a1f780020
:10680000080b20002802880088ff28003802880032
:1068100025608000366080001301c4000000cd00b8
:106820006060880025608000566080001301c4000d
:106830000000cd00c06088006060800008802000fb
:1068400048028800086080005802880011308200e9
:106850008100e90018608000001c78001860880042
:106860000a3082000218c300018009005e18c400cb
:106870000500cd004560880095608000a66080001e
:106880001301c4000000cd00d0608800d5608000f6
:10689000c660800006804200d0608800089020001a
:1068a00048028800786080005802880031308200f9
:1068b0008100e90088608000001c78008860880002
:1068c0002a3082000218c300018009005e18c4004b
:1068d0000500cd00b56088000061800008a02000a0
:1068e00048028800e8608000580288005130820029
:1068f0008100e900f8608000001c7800f8608800e2
:106900004a3082000218c300018009005e18c400ea
:106910000000cd00106188004f0578004f0478001a
:106920004f037800cf0278003600f9003400f900f8
:106930004400f9004a00f9004800f9004600f90057
:1069400000000000000006000000fa008040eb009c
:106950000040eb00050007008040eb0010c0b300d2
:10696000020007000080fa00000006000400fa00a0
:106970002047980031479800d322a9000004200046
:106980004012880040c2bf00614060000004e00087
:10699000fcff320040128000004f78002e40900033
:1069a0000080fb004012880040c2bf0061406000d0
:1069b0000004e000fcff320040128000004f78002d
:1069c0003e4090000080fb004012880040c2bf00a3
:1069d000614060000004e000fcff320040128000d3
:1069e000004f7800d322a8000080fa0000000600c3
:1069f0000400fa0020479800d322a900401280002a
:106a0000004f7800100420004012880040c2bf00f0
:106a1000614060000004e000fcff32002e40900066
:106a20000080fb004012880040c2bf00614060004f
:106a30000004e000fcff32000000eb004012880080
:106a400040c2bf00614060000004e000fcff320073
:106a500040128000004f780040c2bf0061406000db
:106a60000004e000fcff32000000eb004012880050
:106a700040c2bf00614060000004e000fcff320043
:106a800040128000004f7800d322a8001e80fb0037
:106a90000080fa00000006000000fa00d0c2a90041
:106aa00000000000d102a90000000000d122a900ce
:106ab00000000000816a20009140780000ceb30001
:106ac00000c060007041b300a8e6b70000000000fd
:106ad000616d20009140780000ceb30000c06000de
:106ae0007040b300d6e6b70000000000816d2000c2
:106af0009140780000ceb30000c060000034a000d8
:106b0000d8e6b70000000000212420009140780062
:106b1000c0cfb30000c060000014a00042e2b70084
:106b20000000000042c2bf00c041b30042e2b70013
:106b30000000000042a2a8000000000042c2a9001c
:106b40000000000042e2a900000000004302a8008b
:106b5000000000004322a900000000004342a900f9
:106b6000000000004362a900000000004382a90069
:106b7000000000004422a8000000000045a2a80078
:106b80000000000045c2a9000000000045e2a90085
:106b90000000000041a2a9000000000041e2a8009e
:106ba0000000000040c2a90000000000d322a8009d
:106bb0000080fa00000006000a00fa003007980082
:106bc0003e00900002402000110009000200d800a1
:106bd000200798003e0090000240200011000900ac
:106be0000200d8008000fd00100798002e009000e1
:106bf000400798004e009000e10f50001400320052
:106c00004e009000e10f500004003c004e00900048
:106c10000000e00008003200240037004e00900021
:106c2000e20f5000120032004e009000e30f5000bf
:106c3000160032001d0037001e009000800040004a
:106c40004076280000804000100f780017003700c1
:106c5000014020001e009000008050008000400095
:106c60004076280000804000100f78000f003700a9
:106c70001e00900080004000407628000080400008
:106c800010007800000fea000800370001402000e3
:106c90001e009000008050008000400040762800d8
:106ca0000080400010007800000fea001e0078000d
:106cb0000080fa00000006003000fa000e80e800b4
:106cc000016229000e00090031587800f000b1007f
:106cd00071004700116129000e0009003158780049
:106ce000f000b100000220000e00400021602900e9
:106cf0000e00090031587800f000b1000000eb00f0
:106d0000000f780082c0b3008040eb0000c3b300e6
:106d100073fa0700000000000a0037009e007800a8
:106d20000e80e800614178009e0078007100470005
:106d3000e140780000c3b30069fa070000000000da
:106d40001e0fe800e00020009e0f1000f3ff34004b
:106d50000000eb00000f780092c0b3008040eb0011
:106d600000c3b3005efa0700000000000b0037000c
:106d70009e0078000e80e800614178009e00780057
:106d8000000220000e004000e140780000c3b30084
:106d900053fa0700000000001e0fe800e100200089
:106da0009e8f1000f2ff34000080fa000000060001
:106db0003000fa000e80e800e16429000e000900ae
:106dc00031587800f000b10071004700f1632900ec
:106dd0000e00090031587800f000b10000022000d8
:106de0000e004000016329000e00090031587800b0
:106df000f000b1000000eb00000f780082c0b3008b
:106e00008040eb0000c3b30035fa0700000000002b
:106e10000a0037009e0078000e80e800614178008b
:106e20009e00780071004700e140780000c3b30085
:106e30002bfa0700000000001e0fe800e000200011
:106e40009e0f1000f3ff34000000eb00000f7800ed
:106e500092c0b3008040eb0000c3b30020fa0700eb
:106e6000000000000b0037009e0078000e80e80054
:106e7000614178009e007800000220000e00400072
:106e8000e140780000c3b30015fa070000000000dd
:106e90001e0fe800e10020009e8f1000f2ff34007a
:106ea0000080fa00000006003000fa000e80e800c2
:106eb000c16729000e00090031587800f000b100c8
:106ec00071004700d16629000e0009003158780092
:106ed000f000b100000220000e004000e165290032
:106ee0000e00090031587800f000b1000000eb00fe
:106ef000000f780082c0b3008040eb0000c3b300f5
:106f0000f7f90700000000000a0037009e00780033
:106f10000e80e800614178009e0078007100470013
:106f2000e140780000c3b300edf907000000000065
:106f30001e0fe800e00020009e0f1000f3ff340059
:106f40000000eb00000f780092c0b3008040eb001f
:106f500000c3b300e2f90700000000000b00370097
:106f60009e0078000e80e800614178009e00780065
:106f7000000220000e004000e140780000c3b30092
:106f8000d7f90700000000001e0fe800e100200014
:106f90009e8f1000f2ff34000080fa00000006000f
:106fa0003000fa000e80e800a16a29000e000900f6
:106fb00031587800f000b10071004700b169290034
:106fc0000e00090031587800f000b10000022000e6
:106fd0000e004000c16829000e00090031587800f9
:106fe000f000b1000000eb00000f780082c0b30099
:106ff0008040eb0000c3b300b9f9070000000000b7
:107000000a0037009e0078000e80e8006141780099
:107010009e00780071004700e140780000c3b30093
:10702000aff90700000000001e0fe800e00020009c
:107030009e0f1000f3ff34000000eb00000f7800fb
:1070400092c0b3008040eb0000c3b300a4f9070076
:10705000000000000b0037009e0078000e80e80062
:10706000614178009e007800000220000e00400080
:10707000e140780000c3b30099f907000000000068
:107080001e0fe800e10020009e8f1000f2ff340088
:087090000080fa000000060078
:020000040000fa
:10709800b0180000080000000000000000430000d5
:1070a80000040000000000000008000000050000c7
:1070b80000000000c01800000600000000000000ea
:1070c8006418000022000000000000003c180000c6
:1070d8002800000000000000cc180000020000009a
:1070e80000000000a41800000c00000000000000d0
:1070f800b81800000800000000000000c6180000d2
:107108000600000000000000000d0000000b000059
:1071180000000000003e0000000200000000000027
:10712800861800001e000000000000000018000083
:107138003c00000000000000ce1800000200000023
:0871480000000000000000003f
:020000040000fa
:107150000000fa000000eb00001488000000eb00c3
:10716000c01488000000eb00d01488000000eb0081
:10717000e01488000000eb00f01488008142a800b1
:107180000000eb00201488000128200091407800c6
:10719000c0cfb30000c0600080e2b7008102a80049
:1071a0008122a90011148000f0e12f00008060000e
:1071b00001022000010070001014880080c2a900a4
:1071c00080a2a80082c2bf00f040b30082e2b700f4
:1071d0003000200040148800300020006014880037
:1071e000312820009140780030cfb30000c060000b
:1071f0000024a00083e2b70081e2a8000080fa002a
:10720000000006003600f800809fbe00829fbe008e
:10721000849fbe00869fbe003400f800000020005e
:10722000a00188000000fa0038fb07009bf507006a
:107230000000eb00d0c3880010c680000000e8000a
:1072400010c6880010c68000e60f500002003a0009
:107250000000eb0010c688008460a9009460a900bb
:107260000080fa003400f9004f03be004f02be0058
:107270004f01be004f00be003600f900004006007e
:107280000000fa0042c0bf007f40600042e0b7004b
:1072900081e0a900210c20009140780080cfb3004c
:1072a00000c060006040b300c2e0b7008b80a9005e
:1072b0009b80a800d10a200091407800f0c8b3005c
:1072c00000c0600001c4b30001407000ade0b70031
:1072d0008660a9009660a8000080fa000000060001
:1072e0000000fa000421a900000000000441a900e8
:1072f000000000004110200091407800f0ccb30065
:1073000000c0600004e1b7000000000004c1a90053
:107310000000000005a1a900a580a900a5a0a90062
:10732000a5c0a800200020001008880005e1a800e2
:107330008460a9000080fa0000000600801f780029
:107340003400f80000002000a00188000000fa00ce
:107350008660a9009660a9001000200060c6880021
:107360009660a8000080fa003400f9004f00780011
:0473700000400600d3
:020000040000fa
:047374000000fe0017
:00000001FF
